S123B6008E00FFCE1000BDB6D986C3A7391C07FF1D09FF1C2688860097109711971297130D
S123B6209716BDB717206B96148102250A1E00020696188175221A1F00011696101F0804DA
S123B6402D1F08083296111F0810351F08203A20419614810225411C0010BDB736BDB77A0C
S123B660BDB7A1BDB77A1D0010BDB6D9202481FF27267C0010201B8100271D7A00102012F1
S123B68081FF27147C001120098100270B7A001120008D098D43208FBDB717208A1418FF62
S123B6A0BDB7DA8D2B8610A7301F3080FCA6319715A632971481002712DC153CDE1302DF89
S123B6C017389615911425031418FF8D1596183918CE0800180926FC3918CE6000180926F4
S123B6E0FC391D00E096148102252B96188120250E8145250F816025108175251120141C89
S123B700008020121C00C0200D1C004020081C006020031C002039BDB6D91C0080BDB6D99E
S123B7201C0040BDB6D91C0020BDB6D91C0010BDB6D91D00F0391419FFBDB7F68D12BDB76E
S123B740EF8D0D961B9710961A9711961C971239860197118D1096188115250978001196BB
S123B76011810026EF39860197108D56811525097800109610810026F13996148102251EA1
S123B7801419FF961148971D7400118D358115250D7C00119611911D26F1961A97118D3AAF
S123B7A0391419FF961048971E7400108D148115250D7C00109610911E26F1961B97108DB3
S123B7C01939BDB69D9119220E97199610971B9611971A9612971C9618399610A703961190
S120B7E0A7049612810127048D0C20028D01391412011C0008391512011D000839BC
S9030000FC
